:020000020000FC
:1000000012C0189518951895189518951895189563
:100010001FC62BC6189518951895189518951895FC
:100020001895189518950FE50DBF04E00EBF00EA6E
:1000300001BF0FEC08BB0CE207BB0EE304BB00E002
:1000400005BB0AEF01BB05E002BB00EC07B906E007
:1000500006B90AEFD0D5919A949A002700936000D0
:10006000939A06B3037C10B31470012B013CC9F4BE
:1000700005E0C1D506B3037C10B31470012B013C1D
:1000800081F406B3037C10B31470012B073CC9F74D
:1000900001E000937700002700937C0000937D002F
:1000A00030C0E0E0F0E0BDD510937700E1E0F0E093
:1000B000B8D510937C00E2E0F0E0B3D510937D005A
:1000C000E3E0F0E0AED510937E00E4E0F0E0A9D5E7
:1000D00010937F00E5E0F0E0A4D510937800E6E00F
:1000E000F0E09FD510937900E7E0F0E09AD5109307
:1000F0007A00E9E0F0E095D5133008F0112710936D
:100100006000E8E0F0E08DD51B3818F4123108F0FB
:1001100001C012E41093A3020AE00093A80200E0D9
:100120000093A7020093A0020093A1020093A202F1
:100130000093A90206B3037C10B31470012B073C93
:10014000C9F704E009BF02E50DB9709A2AE01AD593
:100150002A95E9F7C29800E000936D0000E0009353
:100160006E0000E000936F0000E00093700000E07C
:100170000093710011D51F3F59F0113019F00AE0BA
:1001800036D5F8CF01E000936D0006D51130E9F3C4
:10019000C29A00E50DB9709A1F3F19F401E0002ED4
:1001A000FEC0D7D3112319F002E0002EF8C00FEFE4
:1001B00073D3112319F403E0002EF1C010937600DD
:1001C00000917700002319F401E00093770064D3D5
:1001D00000919C0010917800011761F400919D003E
:1001E00010917900011731F400919E0010917A006E
:1001F000011741F001E000937700112710937C0074
:1002000010937D006AD2FF93EF93E153F140EF9199
:10021000FF9110F005E023C0FF93EF93ED51F14003
:10022000EF91FF9110F004E01AC0FF93EF93E950B3
:10023000F140EF91FF9110F003E011C0FF93EF93B5
:10024000E55FF040EF91FF9110F002E008C0FF93EE
:10025000EF93E15EF040EF91FF9160F001E0002E3E
:10026000939806E9C8D4939A06E9C5D40A94C1F7CD
:100270004091A50200E80DBD00E00CBD03E00EBDFD
:1002800078940091770010917600101752F401E0F5
:1002900000937700473429F03091600031300AF440
:1002A00036C082D0F89400E00EBD112399F01AF404
:1002B00004E0002E74C011241394012C64D24091E8
:1002C000A502473459F04738A1F0433C01F10091B1
:1002D0007700E7CF00916000023029F000917700AD
:1002E000039500937700112710937C0010937D00F5
:1002F00089CF009177000A9511F400917600009360
:100300007700112710937C0010937D007BCFF89429
:1003100000917700E0E0F0E078D40A2DE1E0F0E031
:1003200074D40B2DE2E0F0E070D4009168000395E6
:1003300003191127080D911EE3E0F0E066D4092DA2
:10034000E4E0F0E062D400917800E5E0F0E05DD414
:1003500000917900E6E0F0E058D400917A00E7E0FF
:10036000F0E053D40091A302E8E0F0E04ED4009115
:100370006000E9E0F0E049D400E010E020E1D8D1ED
:1003800008EC39D4939806B3037C10B31470012B96
:10039000073CC9F70AEF2FD494989198FFCFF894AF
:1003A00011241394F0D1E8CF77D200917700011790
:1003B00011F01FEF0895C0909C00D0909D00E09038
:1003C0009E00F0909F00FF2011F017EF0895C0925B
:1003D0007800D0927900E0927A00A0909A00B090D4
:1003E0009B0022271E2D0D2D1695079508F421E060
:1003F000802E912E6C2C722E30906800A0909A0066
:10040000B0909B0000917C0010917D002227202B52
:10041000212B49F4A0927C00B0927D0080927E0056
:1004200090927F0006C0A02EB12E80907E0090900A
:100430007F000A2D0B210F3F29F0BB2029F402E099
:10044000A01610F41EEF0895B4D152D100270093E6
:10045000A6020093A40201E01127801A910A08F471
:1004600041C0F0926E00E0926F00D0927000C09296
:1004700071005FD30FEF8CD3C0E0D0E080990FC044
:100480006DD04423DAF33FB10FEF0FB92196D2308C
:1004900019F0779BFECFF7CF6AD3142F08953FB1A1
:1004A0000FEF0FB9AC9A48E0330F10F4A99A02C0CD
:1004B000A9980000AD9A4A95AD98AC98A9F72196F5
:1004C000D230E1F654D33A9431F002E01127D00E45
:1004D000E11EF11EC0CF84D1A42CB52C3090680051
:1004E00068D1B9CF062D072911F411270895F0928C
:1004F0006E00E0926F00D0927000C092710019D32C
:100500000FEF46D3C0E0D0E080990FC027D044233E
:10051000DAF33FB10FEF0FB92196D23019F0779B84
:10052000FECFF7CF24D3142F08953FB10FEF0FB9AB
:10053000C615D70568F4AC9A48E0330F10F4A99AB1
:1005400002C0A9980000AD9A4A95AD98AC98A9F759
:100550002196D230C9F60BD311270895F89400E004
:100560000EBDE091A702F091A802319729F0E09327
:10057000A702F093A80220C000E00093A7020AE0BF
:100580000093A802AAD0FF93EF93E35CF040EF91B1
:10059000FF9190F401E02FD3A0D0FF93EF93E35CA1
:1005A000F040EF91FF9140F40AE0002E1124EBD0CF
:1005B00003EC0093A50243C003E01DD336B3337CA4
:1005C00020B32470322B373C21F00091A402031792
:1005D00031F03093A40200270093A6022EC0309180
:1005E000A6023395393119F03093A60226C0009344
:1005F000A50233273093A4023093A602053C39F4B8
:100600001091A3021450123198F412E111C0063C6B
:1006100039F41091A3021C5F1A3850F01AE808C090
:10062000073411F441E00CC0073891F442E008C0EF
:100630001093A3020BE0212F7BD04FEF01C043E0CA
:1006400000E80DBD00E00CBD789403E00EBD0895F8
:10065000033C99F708ECCFD236B3337C20B3247037
:10066000322B333C61F306E4C6D200E002BF01E066
:1006700009BF05E003BF789436B3337C20B3247000
:10068000322B353C99F404E6B6D236B3337C20B332
:100690002470322B353C51F4009160000A950AF425
:1006A00002E00093600044274093A90236B3337CF4
:1006B00020B32470322B333CF9F602E39CD236B3DC
:1006C000337C20B32470322B333CB1F6939AF894E8
:1006D00000E003BF04E009BFB0CF379A349A369ADE
:1006E000349BFECFE4B1F5B13798F695E7950895C0
:1006F000849805E080D2849A00E010E024E018D0CD
:1007000001E079D2809BF4CF00E010E020E010D02F
:1007100003E018E920E00CD00BE01091A302212F98
:1007200007D0E8E4FCE01BD0E8E4FCE018D0089532
:10073000AB9832E008D0302F06D0312F04D0322FC2
:1007400002D0AB9A089548E0330F10F4A99A02C082
:10075000A9980000AA9A4A95AA98B1F7089558E076
:10076000809BFECF3591AC9A48E0330F10F4A99AE4
:1007700002C0A9980000AD9A4A95AD98AC98A9F727
:100780005A9571F70895B4DF112019F0E0E3FCE009
:1007900002C0E8E3FCE0E3DF04E62DD2E0E4FCE0A5
:1007A000DEDF0EE128D20A9479F7E0E4FCE0D7DF3F
:1007B0000895CC24D0906200E0906300F090640033
:1007C0000A2D1B2D025010402227039DD00CE11C46
:1007D000F21E139DE00CF11CDD0CEE1CFF1C0895B5
:1007E00000271091690020916A003327110F221F02
:1007F000331FCA2CDB2CEE24CC0CDD1CEE1CFF249A
:100800000C0D1D1D2E1D3F1DEFEFF1E0E023F12328
:10081000E056FF4F00271E7FC090A002D090A1029B
:10082000E090A202C11621F4D21611F4E31671F081
:1008300030936E0020936F0010937000009371004E
:1008400010D0112319F044245524089501911081EA
:100850001F3F21F4083F12F00FEF1FEF402E512EE3
:10086000089567D1112309F00895A0EAB0E08AD174
:100870001D93A03AE1F7B230D1F779D130916E00F3
:1008800020916F00109170001093A0022093A1029C
:100890003093A20211270895402F5527CC24D090E1
:1008A0006600E0906700FF24DD0CEE1CFF1CF09258
:1008B0006E00E0926F00D0927000C0927100A09024
:1008C0006B00B0906C00EE27FF27EA15FB05FAF5E8
:1008D00030D1112311F0152F089560E1A0E8B0E0A8
:1008E000C0EAD0E04FD11D93AC17BD07D9F70091F6
:1008F0008000002359F1053EC9F000919A00109143
:100900009B00012B99F000918B00087179F4009104
:1009100088000D3459F400918900003539F40091B4
:100920008A00033319F453954A9581F031966A95FC
:10093000A9F61DD102E01127D00EE11EF11EF092A2
:100940006E00E0926F00D0927000BFCF10D1152FD3
:10095000089500E00093720000E00093730001E04E
:10096000009374000EEB00937500B4D020908800C3
:10097000309089000027122D232D3327110F221FBD
:10098000331F309372002093730010937400009310
:100990007500A0D000918B0010918C001F930F93D5
:1009A000005012400F911F9111F012E00895009134
:1009B0008D000093680000918E0010918F00020D51
:1009C000131D0093690010936A000091910010912B
:1009D000920000936B0010936C00A0909600B09072
:1009E0009700AA2021F4BB2011F411E00895209172
:1009F0009000A29E112D002DB29E100D2091690035
:100A000030916A00020F131F009366001093670075
:100A100000916B0010916C001295212F207F1F70A8
:100A20003FE0302302950F70022B332311F00F5F4C
:100A30001F4F209166003091670000241124200F81
:100A4000311F011C20936200309363000092640008
:100A50001092650000919300109194002227332793
:100A6000FF24F12AF02AB1F400E2FF24220C331C07
:100A7000FF1CF09272003092730020927400009379
:100A8000750028D000918000109181002091820093
:100A900030918300D0906900E0906A00FF240D1926
:100AA0001E092F093F09442750916800652F529570
:100AB000507F62956F707727041715072607370751
:100AC00012F001E003C0002713E0089500936100D5
:100AD00011270895F0907200E0907300D090740098
:100AE000C09075003F2D2E2D1EEF1D210027309345
:100AF0006E0020936F00109370000093710019D066
:100B0000112309F008952C2D31E03D21CC27DD275C
:100B1000A0E8B0E0E0EAF0E035D0C217D30722F059
:100B2000AE17BF070AF41D932196D230A9F71FD044
:100B3000089534E6C29801E100936D002DD0112391
:100B400051F4A0E0B0E11ED01E3F11F4112708952A
:100B50001197C9F704C01E3F11F411270895C29AD6
:100B600004E145D03A9509F0E5CF11E008950AD0A7
:100B700009D0C0E0D8E006D01F3F11F02197D9F787
:100B8000C29A08950FEF0FB9779BFECF1FB108955A
:100B90000FB9779BFECF0895C0E0D8E0F3DF1F3F89
:100BA00021F02197D9F711E0089500916D00102FE1
:100BB0000064EEDF00916E00EBDF00916F00E8DF74
:100BC00000917000E5DF00917100E2DF112311F464
:100BD00005E901C001E0DCDFC0E0D8E0D3DF1E3F63
:100BE00029F020E8212311F02197C1F70895000092
:100BF0000A95E9F7089512E323E100002A95E9F741
:100C00001A95D1F70A95B9F708950BD0011709F491
:100C10000895E199FECFFFBBEEBB0DBBE29AE19ACE
:100C20000895E199FECFFFBBEEBBE09A1DB3089596
:100C300053EF6E310000000053EF6E3500000000EE
:100C4000457869740000000000000000000000000A
:100C50000FE50DBF04E00EBF009177001127109340
:100C60007C0010937D0078941CCB0FB6E09160005F
:100C7000F3E0EA9512F0FF0FFCCF4091A9024395F3
:100C80004F1731F44427939902C0939A01C0939867
:080C90004093A9020FBE189564
:00000001FF
